:02000000072DCA
:08000800FF00030E8316031331
:10001000A0000A0EA100040EA2008A110A123B2DB4
:1000200000000000BB0B10280800BA08031D1928A7
:100030000800F9300000000000000000000000008F
:1000400000000000000000000000000000000000B0
:1000500000000000FF3E031D1A2800000000000001
:100060000000000000000000000000000000000090
:10007000000000000000000000000000BA0B19287A
:100080000800BE08031D4528080009300000FF3E97
:10009000031D462800000000BE0B4528080005117E
:1000A0008312051101308316BB0010203918051585
:1000B0003C30BB00102005150A30BB0010200800A2
:1000C0008316031305118312051101308316BB003B
:1000D000102005150A30BB001020043083120505DE
:1000E0008316BA003230BB0010203A08BB0008006B
:1000F000C101C201C401C501C301431A08000310B4
:10010000C40DC50DBB0DBC0DC10DC20D3E08420294
:10011000031D8C283D084102031C95283D08C1029F
:100120003E08031CC203C2024414C30A7D28B9015D
:10013000380839020318080064000130BA0015209D
:10014000B90A98289C18A2283A089B003C089A00F3
:100150001C1580300B05BD008B1355309D00AA3057
:100160009D009C149C18B228BD080319B8288B1751
:100170001C110800BA0138089B001C141A08BA00A8
:100180003A08BB00080083160313B701B801B90190
:10019000083037020318DB2860203B08B900B80894
:1001A0000310B80C3908003C0318D92880303804F3
:1001B000B800B70AC8283808BA000800B8010830E3
:1001C0003802031808003708B9004F20B708031099
:1001D000B70CB80ADF28831603130515051183121F
:1001E0000511C8308316BB001020C830BB0010209A
:1001F000C830BB00102005153C30BB001020043077
:10020000831205058316B6003603031D0A29013043
:10021000B70008008C30BB001020C830BB00102095
:10022000C830BB001020B7010800831206108610EA
:10023000061186110612861283163B0E0F39BD0079
:100240000F30BD053D1C2629831206148316BD1CE4
:100250002B298312861483163D1D3029831206151F
:100260008316BD1D3529831286158316BC08031914
:100270003B29831206160A308316BE0041208312E2
:1002800086160A308316BE004120831286120F3074
:1002900083163B05BD000A30BE00412083120610C4
:1002A0008610061186110612861283163D1C5A29E5
:1002B000831206148316BD1C5F29831286148316CD
:1002C0003D1D6429831206158316BD1D69298312FD
:1002D00086158316BC0803196F29831206160A3087
:1002E0008316BE004120831286160A308316BE0094
:1002F0004120831286120A308316BE004120080076
:10030000FF3083160313B5008515083083120505E9
:100310008316B5003508B6000800FF3083160313B6
:10032000B70005140130831205058316B70037089E
:10033000B8000800FF3083160313B700851402309D
:10034000831205058316B7003708B800080083122A
:10035000031361088316B400B501B6013408B70071
:100360003608B4003708B500831260088316B40459
:10037000B5083408B6003508B70008008316031323
:10038000B501EB20B7080319C8290130B6000800F1
:10039000CC30B700DE20BE30B700DE200930350299
:1003A0000318E029C3203A08B40083128313603095
:1003B000840083163508840734088000B50ACE29E6
:1003C000B601080083160313B401B501EB20CC304D
:1003D000B700DE204430B700DE20B408031DFD293D
:1003E000C3203A08B4000430BA001520B50A350A13
:1003F000031DED290130B6000800B6010800B71F43
:100400000E2A2D30BB001030BC0015213608003CF0
:10041000BB00B7090318B70A3B08B6003608B80096
:100420003708B90027303702031D182A103036026A
:10043000031C462AB71B462ABF013808BB003908EF
:10044000BC00B91F292ABB09BC09BB0A0319BC0A95
:10045000BF0A1030BD002730BE0078204408BA0023
:100460003F1C342ABA09BA0A3A08303EBB001030A1
:10047000BC0015213A08003C0318462A1030B80287
:100480002730031C2830B902BA033A2A0330370256
:10049000031D4C2AE8303602031C7C2AB71B7C2A39
:1004A000C0013808BB003908BC00B91F5D2ABB0970
:1004B000BC09BB0A0319BC0AC00AE830BD000330FE
:1004C000BE0078204408BF00401C682ABF09BF0A4C
:1004D0003F08BA003A08303EBB001030BC0015217E
:1004E0003A08003C03187C2AE830B8020330031CA9
:1004F0000430B902BA03702A3708803ABB00803052
:100500003B02031D852A64303602031CB12AC00158
:100510003808BB003908BC00B91F942ABB09BC09C4
:10052000BB0A0319BC0AC00A6430BD00BE017820B2
:100530004408BF00401C9E2ABF09BF0A3F08BA00FA
:100540003A08303EBB001030BC0015213A08003C90
:100550000318B12A6430B802B908031CB903BA03FE
:10056000A62A3708803ABB0080303B02031DBA2A16
:100570000A303602031CE62AC0013808BB003908DD
:10058000BC00B91FC92ABB09BC09BB0A0319BC0AB4
:10059000C00A0A30BD00BE0178204408BF00401CDC
:1005A000D32ABF09BF0A3F08BA003A08303EBB0051
:1005B0001030BC0015213A08003C0318E62A0A3026
:1005C000B802B908031CB903BA03DB2A3808303E65
:1005D000BB001030BC00152108003608BB001030ED
:1005E000BC0015210800B708031DF92A8030B700A8
:1005F000FB2AC030B70036083707BB00BC01152105
:100600000230B800972008003608BA003708BB004F
:100610003808BC00A22008003608B8003708B90026
:10062000BA203B08B800B90108007F3083160313D5
:10063000060586007F30831206058316B4008030DD
:10064000340483128600E2213608AE00BE2136084B
:10065000AE00A7213608A3003708A4007F300605A6
:1006600086007F308312060586008316A30E0F30A6
:10067000A305240EA400F039A3040F30A405013013
:10068000B600B701F3222030B600ED227430B60078
:10069000ED226530B600ED226D30B600ED227030EF
:1006A000B600ED222030B600ED223D30B600ED223E
:1006B0002030B600ED222308C83C03182408031993
:1006C000802BBF3006058600BF30831206058316D7
:1006D000B400403034048312860083162308003CA3
:1006E000B4002408031C240A103CB5003408A300FD
:1006F0003508A4000130B1002D30B600ED22812B69
:10070000B1012308B6002408B700FF212030B6004D
:10071000ED224330B600ED222030B600ED2220302D
:10072000B600ED222030B600ED222030B600ED22DA
:100730002030B600ED220800831603132F08320282
:10074000230224080318B22B031DB22BBF30060569
:100750008600BF30831206058316B600403036048B
:10076000831286008316B501320823022408031879
:10077000BB2B0319BC2BB50AB401B40AB108031D85
:1007800034103408350503190800BF30060586000B
:10079000BF30831206058600080083160313B601D6
:1007A000B7010C233808B2009A21B601B808031D1E
:1007B000361430103608031D3014301CEA2BC830B4
:1007C000BA001520320AB200B601B7013208B800EB
:1007D000B90104238D21B601B808031D3614B010E9
:1007E0003608031DB014B01C002CC830BA00152008
:1007F0003203B200B601B7013208B800B9010423D0
:10080000320A031D0A2CB201B601B7013208B80042
:10081000B9010423B5017D3032020318B50AB401D1
:10082000FF303202031CB40A340835050319202CAA
:100830007D30B200B601B7013208B800B901042317
:100840000130B600B700F3227230B600ED2220303E
:10085000B600ED223D30B600ED222030B600ED228C
:100860003208B600B701FF212030B600ED22433038
:10087000B600ED222030B600ED222030B600ED2289
:100880006730B600ED223D30B600ED222F08B600ED
:10089000B701FF212030B600ED222030B600ED2256
:1008A0002030B600ED220800013083160313B60095
:1008B000B7010C233808AF008021B401B608031D2E
:1008C000341430113408031D3015301D732CC8301A
:1008D000BA0015202F0AAF000130B600B7012F086B
:1008E000B800B90104232F08053C031808000130A3
:1008F000AF00B600B7012F08B800B9010423080003
:1009000083160313B601B7010C233808B20032086E
:100910007D3C0318912CB601B7013230B800B90103
:1009200004230130B600B7010C233808AF002F08AC
:10093000053C031808000130B600B7010130B800CB
:10094000B90104230800831603130610831206104E
:1009500083168610831286108316061183120611E1
:1009600083168611831286118316061283120612CD
:1009700083168612831286120C308316B8009720D5
:100980003330BB00BC0115210230B8009720333052
:10099000BB00BC0115210230B80097203230BB00EB
:1009A000BC0115210230B80097202C30BB00BC01DF
:1009B00015210230B80097200630BB00BC0115217C
:1009C0000230B80097200C30BB00BC01152102306A
:1009D000B80097200130BB00BC0115210230B800DF
:1009E00097200230BB00BC0115210230B8009720CF
:1009F00008000730831203139F00C0308316810064
:100A0000A324802415239C23CD235424022DD530E8
:100A100083120313E900C430EA00BB30EB00DC3082
:100A2000EC00ED01EE01EF01F001F101F201F30143
:100A3000F401F501F601F701F8018316A801A901F7
:100A4000FD01FE01AA01AB01AC01AD01F901FA0102
:100A5000FB01FC01A601A701A501B30183128313C9
:100A6000203084003F30DF008001840A8A110A129E
:100A7000DF0B342DF92C83160313220E8400210E74
:0C0A80008A00200E8300FF0E7F0E09008C
:02400E00023F6F
:00000001FF
